:0200000480007A
:100000009710000093800000171100001301810277
:1000100083A1000013020000930210001303F0FFFD
:10002000B70300809383F3FF3704008033C241009D
:10003000B3C2510033C36100B3C3710033C4810044
:100040002320310023224100232451002326610074
:1000500023287100232A8100971000009380C0FAA2
:1000600017110000130181FE03A400009304000097
:10007000130510009305F0FF370600801306F6FF06
:10008000B7060080B34494003345A400B345B400E0
:100090003346C400B346D4002320810023229100BC
:1000A0002324A1002326B1002328C100232AD10044
:1000B00097100000938080F517110000130181FA5A
:1000C00083A6000013070000930710001308F0FF39
:1000D000B70800809388F8FF3709008033C7E6002F
:1000E000B3C7F60033C80601B3C8160133C92601E9
:1000F0002320D1002322E1002324F1002326010143
:1001000023281101232A210197100000938040F039
:1001100017110000130181F603A9000093090000E4
:10012000130A1000930AF0FF370B0080130BFBFF3C
:10013000B70B0080B3493901334A4901B34A590129
:10014000334B6901B34B7901232021012322310173
:10015000232441012326510123286101232A71010F
:1001600097100000938000EB17110000130181F23B
:1001700083AB0000130C0000930C1000130DF0FF74
:10018000B70D0080938DFDFF370E008033CC8B01BF
:10019000B3CC9B0133CDAB01B3CDBB0133CECB018F
:1001A0002320710123228101232491012326A1010F
:1001B0002328B101232AC101971C0000938CCCE5B0
:1001C000171D0000130D8DEE03AE0C001302F00797
:1001D0009302F0031303F0019303F0001304700083
:1001E00093043000B34E4E0033CF5E00B34F6F0028
:1001F000B3C07F0033C18000B341910023204D0084
:100200002322CD012324DD012326ED012328FD0136
:10021000232A1D00232C2D00232E3D0097100000C3
:100220009380C0DF17110000130141EA03AE000004
:10023000B79DFFF7938D8D813340BE0123200100D0
:10024000971000009380C0DD17110000130141E8F2
:1002500003AE0000B79DFFF7938D8D813340BE0143
:10026000B342000023200100232251009710000018
:10027000938040DB17110000130101E683A1000009
:1002800033C20100B342020033435000334703003E
:10029000B347070033C80700B34C0001334D90014A
:1002A000B34D0D00232041002322A1012324B101DD
:1002B00017150000130505D897150000938585E2F2
:1002C000370610F01306C6F26306B5028326C50092
:1002D0002320D600832685002320D60083264500D0
:1002E0002320D600832605002320D6001305050110
:1002F0006FF09FFD370510F0130505F22320050070
:0403000000000000F9
:101000000000000001000000FFFFFFFFFFFFFF7F67
:1010100000000080FFFFCDAB7856341298BADCFE9A
:10102000145892360000000000000000000000008C
:10103000FFFFFFFFFFFFFFFFFFFFFFFFFFFFFFFFC0
:10104000FFFFFFFFFFFFFFFFFFFFFFFFFFFFFFFFB0
:10105000FFFFFFFFFFFFFFFFFFFFFFFFFFFFFFFFA0
:10106000FFFFFFFFFFFFFFFFFFFFFFFFFFFFFFFF90
:10107000FFFFFFFFFFFFFFFFFFFFFFFFFFFFFFFF80
:10108000FFFFFFFFFFFFFFFFFFFFFFFFFFFFFFFF70
:10109000FFFFFFFFFFFFFFFFFFFFFFFFFFFFFFFF60
:1010A000FFFFFFFFFFFFFFFFFFFFFFFFFFFFFFFF50
:1010B000FFFFFFFFFFFFFFFFFFFFFFFFFFFFFFFF40
:1010C000FFFFFFFFFFFFFFFFFFFFFFFFFFFFFFFF30
:1010D000FFFFFFFFFFFFFFFFFFFFFFFFFFFFFFFF20
:040000058000000077
:00000001FF
